:020000040800F2
:10000000381A00200501000811300008D129000825
:10001000192D0008750D0008B1400008000000000F
:10002000000000000000000000000000593500083A
:10003000BD14000800000000113400085B35000802
:100040001F0100081F0100081F0100081F01000810
:100050001F0100081F0100081F0100081F01000800
:100060001F0100081F0100081F0100081F010008F0
:100070001F0100081F0100081F0100081F010008E0
:100080001F0100081F0100081F0100081F010008D0
:100090001F0100081F0100081F0100081F010008C0
:1000A0001F0100081F0100081F0100081F010008B0
:1000B0001F0100081F0100081F0100081F010008A0
:1000C0001F0100081F0100081F0100081F01000890
:1000D0001F0100088140000891400008A14000086D
:1000E0001F0100081F0100081F010008DFF810D0E1
:1000F00000F0C8FB00480047C14D0008AFF3008086
:10010000381A00200648804706480047FEE7FEE709
:10011000FEE7FEE7FEE7FEE7FEE7FEE7FEE7FEE7B7
:10012000CD350008ED000008202A04DB203A21FA32
:1001300002F00021704721FA02F3D040C2F1200200
:10014000914008431946704700487047585E0008C0
:1001500010B50446FFF7F8FF0068005D00F00100ED
:1001600010BD40EA01039B0703D009E008C9121F34
:1001700008C0042AFAD203E011F8013B00F8013B61
:10018000521EF9D27047D2B201E000F8012B491E8D
:10019000FBD270470022F6E710B513460A46044624
:1001A0001946FFF7F0FF204610BD421C10F8011B56
:1001B0000029FBD1801A704710B5002200E0521CC4
:1001C000835C8C5CA34201D1002BF8D1D8B2E1B2A0
:1001D000401A10BD30B505460020034600E05B1C08
:1001E000934205D2EC5CC85C201A01D1002CF6D1F8
:1001F00030BD00000FB400B58DB010A909900B9070
:1002000000914FF0FF300A9000200C9005480690B6
:10021000054807906A4609A80F9900F015F90DB036
:100220005DF814FB65040008830400082DE9FF5FF6
:100230001D464FF0FF3BD5E9014691465F464FF022
:100240000008A9697F1C01988847296A8246884767
:100250000028F6D1BAF1FF3F0CD024F4C064002E80
:1002600019DD600614D5BAF12B0F09D0BAF12D0FA4
:100270000ED103E0584604B0BDE8F09F44F480641A
:10028000A9697F1C01988847761E8246002E02DDF0
:10029000BAF1300F03D0B9F1000F26D032E0A969CE
:1002A000761E44F400747F1C019888478246002E15
:1002B00005DDBAF1780F06D0BAF1580F03D0B9F1C5
:1002C000000F10D01EE0B9F1000F02D0B9F1100FED
:1002D00018D1A969761E24F400747F1C0198884700
:1002E0008246102002E0082000E00A20814609E052
:1002F00008FB0908A969761E44F400747F1C019864
:1003000088478246002E05DD4946504600F088F8B1
:100310000028EDDAE96901988847A00502D46FF05A
:100320000100A8E7E00725D1600613D5600502D5D6
:10033000C8F1000000E0404629680A1D2A600968EB
:10034000220501D5087015E0220701D5088011E0CB
:1003500008600FE02868011D29600068210502D5AA
:1003600080F8008006E0210702D5A0F8008001E0B7
:10037000C0F8008038467EE770B5064603F0FAFE06
:10038000046805460A220021304600F08BF82C60F4
:1003900070BD30B50B46014600202022012409E043
:1003A00021FA02F59D4205D303FA02F5491B04FA2E
:1003B00002F52844151EA2F10102F1DC30BD2DE941
:1003C000F05F0546002092469B46884606468146D9
:1003D00040241BE02846414647462246FFF7A4FE3C
:1003E00053465A46C01A914110D311461846224628
:1003F00000F05AFA2D1A67EB01084F4622460120F9
:10040000002100F051FA17EB00094E41201EA4F123
:100410000104DFDC484631462A464346BDE8F09FEA
:100420003A2800D2303820F02002412A01D3A2F12C
:100430003700884201D34FF0FF3070470268114403
:100440001378016018467047D1600449516104492E
:10045000116200211161114600F048BA3D04000804
:1004600051010008426842B1016811F8013B23B113
:10047000521EC0E90012184670470121C160881E53
:10048000704742685AB1C368016843B983688B42B8
:1004900005D0491E521CC0E90012002070474FF0E1
:1004A000FF3070472DE9F04791460F4680460446DD
:1004B000002614F8015B2DB1FFF746FE0068405D91
:1004C000C007F6D12B2D02D02D2D18D0641E4A4620
:1004D0003946204600F0A2FB27B13968A14201D17C
:1004E000C7F8008071054FF002040BD54042002888
:1004F00003DD03F03FFE0460A007BDE8F08746F48B
:100500008066E4E70028F8DA03F034FE04606FF058
:100510000040F2E72DE9FE4F804681EA0300C00F5C
:100520000C46009021F0004123F00045B8EB02009A
:10053000A94105D24046214690461C460B4602463C
:1005400023F00040104347D0270DC7F30A00C3F340
:100550000A510290401A019040286BDAC3F313004D
:1005600040F4801B0098924620B10023D2EB030A8E
:1005700063EB0B0B01985946C0F14002504600F066
:1005800093F906460D4650465946019A00F09BF9EC
:1005900010EB08006141002487EA115284EAE773F6
:1005A0001A4340D0009A62B3019A012A4FEA0752D7
:1005B00015DC001B61EB02014FF0004202EA07521A
:1005C000CDE90042001C41F5801132462B4600F077
:1005D00083FB03B0BDE8F08F40462146F9E7001BDE
:1005E00061EB0201001C41F5801300185B412018EB
:1005F000A2F5001747EB030140EAD570B6196D412B
:1006000011E06D084FEA360645EAC0754FEA075219
:10061000001B61EB0201001C41F5801149084FEA03
:1006200030000019514132462B4603B0BDE8F04F6F
:1006300000F043BB0098012240000023D0EB0202EF
:1006400063EBE073009821464FEAE074B8EB0000DA
:1006500061EB0401E9E783F000435BE781F00041CF
:1006600058E72DE9FE4F81EA030404F0004421F02D
:10067000004100944FF0000B23F0004350EA0104C6
:100680005ED052EA03045BD0C3F30A54C1F30A55A7
:100690002C44A4F2F3340194A0FB0254C1F31301DF
:1006A00041F48011C3F3130343F4801301FB0244AC
:1006B00000FB034E840A970A44EA815447EA8357B1
:1006C000A4FB076802958D0A05FB07854FEA932C6A
:1006D00004FB0C542705029D4FEA065847EA1637DB
:1006E000B5EB08056EEB070C870E920E47EA8117F3
:1006F00042EA8312A7FB0201B6EB0B0164EB000494
:100700002B0D43EA0C335E1844EB1C50DA4651467D
:10071000E7FB0201C5F313044FEA0B3343EA14531A
:100720004FEA0432019C43EA0603A4F10C0402944C
:10073000009CCDE900B400F0CFFA03B0BDE8F08F23
:1007400000200146F9E72DE9F04D81EA030404F0A9
:10075000004B21F0004514464FF0000A23F0004101
:1007600050EA050220D054EA01021DD0C5F30A5711
:100770000246C5F31303C1F31300C1F30A5640F454
:10078000801543F48013A7EB0608101BD64608F229
:10079000FD3873EB050002D308F1010801E092185F
:1007A0005B41B8F1000F03DA00200146BDE8F08D8F
:1007B00000204FF48011064684460EE0171B73EBB1
:1007C000050705D3121B63EB050306434CEA010C36
:1007D00049084FEA300092185B4150EA0107EDD119
:1007E00052EA030012D082EA040083EA05010843BA
:1007F00005D0101BAB4106D20122002306E00022E7
:100800004FF0004302E06FF0010253101AEB0600B4
:100810004CEB085110EB0A0041EB0B01BDE8F04D29
:1008200000F04BBAC1F30A52C1F3130140F2FF3397
:1008300041F480119A4202DA00200146704740F2EA
:1008400033439A42A2F2334202DC5242FFF76CBCBD
:1008500000F02AB830B5041E71F1000404DB4FF03B
:100860000044404264EB0101141E73F1000405DBF7
:100870001C464FF00043524263EB0403994208BF09
:10088000904230BD064C074D06E0E06840F00103A1
:1008900094E8070098471034AC42F6D3FFF72AFCDF
:1008A000945E0008B45E0008202A04DB203A00FAB7
:1008B00002F1002070479140C2F1200320FA03F3B7
:1008C000194390407047202A06DBCB17203A41FAA3
:1008D00002F043EAE07306E041FA02F3D040C2F1CD
:1008E0002002914008431946704700002DE9F34F5C
:1008F0008BB04FF0000801F10C000C464FF0010BDB
:1009000046460DF1080A019062690121019890475D
:10091000051E2DD0252D2CD0216A8847C0B16269D3
:10092000012101989047216A88470028F7D1411E8C
:1009300062690198904700E0761CA1690B9888478E
:10094000216A88470028F7D1E1690B988847DBE7DF
:10095000A1690B9888470746A84201D1761CD3E7C6
:10096000E1690B9888477F1C02D1B8F1000F6FD066
:1009700047E1002762693D463946019890472A2899
:1009800004D162690121019890470125DFF888921E
:100990006269012101989047A0F130010A290AD229
:1009A0004F45E5DC07EB870100EB4107303FDFD423
:1009B00045F01005ECE7E90601D46FF000476C281C
:1009C0000AD04C2814D0682815D06A280DD0742875
:1009D0001CD07A281AD01DE0626901210198904745
:1009E0006C2802D045F0040514E045F002050DE046
:1009F00045F020050AE062690121019890476828C6
:100A000002D045F0080505E045F400656269012162
:100A100001989047C4E9015765283DD019DC582852
:100A20007AD00CDC452837D004DC252826D0412894
:100A300031D131E046282FD047282CD12CE05B283B
:100A400077D0612828D063287CD0642823D15AE04D
:100A5000D1E06F2848D008DC66281DD067281BD05D
:100A6000692821D06E2816D127E0702845D0732838
:100A700068D0752847D078280DD14DE0A1690B9832
:100A80008847054625283FF469AFE1690B988847F8
:100A90006D1C3FF46AAFB4E023466A466FF0010074
:100AA0000B99AFF300809FE045F040006060A8071D
:100AB00023464FF0000236D43EE0E8077FF447AF0C
:100AC0002068011D21600068290501D506701BE71B
:100AD000290701D5068017E7A90703D5F117C0E953
:100AE000006111E706600FE745F040006060A8076D
:100AF00023464FF0080216D41EE040F60E0125EA08
:100B00000100606016E045F040006060A8072346E1
:100B10004FF00A0207D40FE045F040006060A807DC
:100B200008D5234610226FF001000B99AFF3008027
:100B30005AE007E0234610226FF001000B99FFF7FF
:100B400075FB51E04FF000094F464B46632802D039
:100B50005B2807D041E02079C00601D40120A060C5
:100B600001273AE062690121019890475E2805D18A
:100B70004FF001096269494601989047216939B9E6
:100B800000210A46534643F82120491C0829FADB74
:100B9000B0B3216969B9C11700EBD16253110AEBF7
:100BA000830122F01F02821A01200B689040034348
:100BB0000B6062690121019890475D28E8D1B9F185
:100BC000000F09D00020514651F82020D24341F8AF
:100BD0002020401C0828F7DB02AB224600976FF06C
:100BE00001000B99AFF3008000280CDA401C08D1FB
:100BF000BBF1000F05D04FF0FF300DB0BDE8F08F16
:100C0000FFE74046F9E7E90701D108F1010806448A
:100C10004FF0000B78E60000CCCCCC0C2DE9F05F57
:100C200082460078002715468B460AF10104B94632
:100C3000302801D09DB113E014F8010B012778286A
:100C400003D0582801D045B10AE00DB1102D07D1CD
:100C50000027102514F8010B02E0082500E00A2502
:100C60000026B0460EE005FB080005FB06F1012753
:100C700001EB10461FFA80F8B6F5803F00D3B94665
:100C800014F8010B2946FFF7CBFB0028EBDABBF188
:100C9000000F05D00FB1641E00E05446CBF80040B1
:100CA000B9F1000F06D003F065FA02210160C81EF9
:100CB000BDE8F09F48EA0640FAE710B5141E73F14C
:100CC000000408DA401C41F1000192185B411A430C
:100CD00001D120F0010010BD2DE9F04D92469B4658
:100CE00011B1B1FA81F202E0B0FA80F220329046FE
:100CF000FFF7DAFD04460F4640EA0A0041EA0B011D
:100D000053465A46084313D0114653EA010019D0FE
:100D1000C8F140025046FFF707FA05460E46504616
:100D200059464246FFF7C0FD084305D0012004E0C4
:100D300020463946BDE8F08D0020054346EAE076BE
:100D40002C4337430A986305E40AA0EB080000220D
:100D5000FD0A44EA47540A3002D500200146E9E77B
:100D6000010510196941DDE9084500196941BDE82F
:100D7000F04DA2E700BFFEE770B504460D46B5484A
:100D80000078C8B1B3480078052815D0B148406D47
:100D9000281AB0F57A7F0FD3AE48806D401CAD495C
:100DA0008865ADA002F03CFC04F056FA242C02D178
:100DB0000120A849087070BDA6484565007806283E
:100DC0000BD2DFE800F0030B57A4E2F9242C04D186
:100DD00004F042FA01209F49087037E12C2C0CD115
:100DE00000219C4890F84E20401C815402209949D3
:100DF0000870002081F84E003BE02A2C0ED1002123
:100E0000944890F84E20401C815404209149087069
:100E1000002081F84E0081F852002AE0204603F0BD
:100E2000A9FFF8B18B4890F84E00072812DA8948DC
:100E300090F84E1090F84E00401C864A82F84E0002
:100E4000501C4454401E90F84F006040114681F8F9
:100E50004F000EE07F48806D401C7E49886504F09D
:100E6000FBF906E07B48806D401C7A49886504F0F8
:100E7000F3F9EBE02C2C0CD10021764890F84E20B1
:100E800009308154032073490870002081F84E0016
:100E90003CE02A2C0ED100216E4890F84E200930FB
:100EA000815404206B490870002081F84E0081F8BD
:100EB00052002BE0204603F070FF00B3654890F825
:100EC0004E001F2813DA634890F84E1090F84E0039
:100ED000401C604A82F84E0002F10900445409386F
:100EE00090F84F006040114681F84F000EE05948DD
:100EF000806D401C5749886504F0AEF906E05548FE
:100F0000806D401C5349886504F0A6F99EE02A2CA8
:100F10000ED100214F4890F84E20293081540420F2
:100F20004C490870002081F84E0081F852002BE0F7
:100F3000204603F032FF00B3464890F84E001F28C9
:100F400013DA444890F84E1090F84E00401C414A85
:100F500082F84E0002F129004454293890F84F00DD
:100F60006040114681F84F000EE03A48806D401C09
:100F70003849886504F070F906E03648806D401CF9
:100F80003449886504F068F960E00A2C42D1314A9E
:100F900092F8511092F8500003F07BFE2D4981F831
:100FA0004900084690F84F1080F84A1090F8490020
:100FB000FF2802D1012101E040E00021254880F80E
:100FC0004D1090F84D0030B9224890F8491090F833
:100FD0004A0081420BD101211E4880F84C100520A7
:100FE0001C4908700846C06D401CC86525E01948BA
:100FF000806D401C17498865084690F84A2090F893
:1010000049101DA002F00CFB26A004F06BFD04F0BB
:1010100023F912E00D2C10D00E4890F8520002284F
:101020000BDA0C4890F8521090F85200401C094A14
:1010300082F8520002F15000445407E004F00CF929
:10104000242C02D101200349087000BF00BF00BF5B
:10105000B1E60000340200205B434D445D2054693A
:101060006D656F75742C2072657365742070617284
:101070007365720D0A0000005B434D445D204368B8
:1010800065636B73756D206572726F723A2072655D
:1010900063763D253032582063616C633D253032E4
:1010A000580D0A004353000010B504460948007863
:1010B00005280CD1074890F84C0040B12CB14D22C6
:1010C0000449491C2046FFF74CF8012010BD0020C0
:1010D000FCE700003402002010B560210448FFF74F
:1010E00059F800200249087002A002F099FA10BDD8
:1010F000340200205B434D445D20496E6974204FEB
:101100004B0D0A00014908607047000008000020EC
:1011100001490870704700000C00002010B5074816
:101120000078052809D1054890F84C0028B10348FB
:10113000401C03F0FFFE04F08FF810BD34020020C5
:1011400010B5002018E01A4901EB001108700021C9
:10115000174A02EB00125160154A02EB001291602F
:10116000134A02EB00121173124A22F81010124AAD
:1011700042F82010411CC8B20328E4DB00200F49CC
:1011800008600F4908600F49086001200E49087087
:101190000E48FFF7B7FF02F067FD01F04DFF0CA00E
:1011A00002F03EFA032114A002F03AFA10BD00004A
:1011B000A0030020720000205005002064000020E1
:1011C000680000206C00002070000020B54A000874
:1011D0005B524F555445525D205541525433205374
:1011E0006D61727420526F7574657220656E6162F4
:1011F0006C65640D0A0000005B524F555445525D0A
:1012000020496E6974204F4B2C20256420706F722A
:10121000747320726567697374657265640D0A0082
:1012200070B5A2B000F084FB05460024204601F012
:10123000BBFD0646002E30DD4B4804702046FFF70C
:1012400067FF12E09DF88410204603F0F7FB294663
:101250009DF88400FFF790FD444800EB041080687F
:10126000401C424901EB0411886021A9204601F08D
:1012700009FE0028E6DC0020FFF716FF60B12046DB
:1012800003F052FC3A480068401C394908600120CC
:10129000364901EB0411087300BF2AE029469DF886
:1012A000840002F00BFB044604B3012C02D0022C94
:1012B0001DD10FE00220FFF72BFF29469DF8840087
:1012C000FFF75AFD9DF884302AA22FA1002000F0DC
:1012D0009DF80CE09DF8840001F0BAFF9DF8843081
:1012E0002BA229A1002000F091F800E000BF00BF70
:1012F00000BF21A9022001F0C5FD0028CEDC284650
:1013000002F082FA88B1694601A802F06BFC58B17C
:10131000BDF8001001A801F0F3FEBDF8003021A2D5
:1013200019A1012000F072F800BF02F003F80024B8
:1013300013E0012C00D10EE0224830F81400002800
:1013400008DD214850F82400281A322802D320460C
:1013500003F0EAFB00BF601CC4B2032CE9DBFFF71B
:10136000DDFE22B070BD000070000020A003002050
:1013700068000020434D4420627974653A2030783B
:10138000253032580000000055415254330000000F
:1013900050545820627974653A203078253032589C
:1013A00000000000504153535448524F5547483AAB
:1013B0002025642062797465732071756575656494
:1013C00000000000720000205005002010B5002031
:1013D0000349087003F06CFC02A002F09BF910BDF9
:1013E000780000205B4C4F475D20446562756720A4
:1013F0006C6F672073797374656D20696E697469A9
:10140000616C697A65640D0A000000000FB470B564
:10141000C2B005460E4622480078854203DA42B043
:1014200070BC5DF814FB304603F05EFC00B9F6E7D3
:1014300000240EB1304600E01AA01C4A009052F879
:101440002530C4F5807102AA101919A202F042FEDB
:101450000444FF2C0DDA49A80190C4F5807102AA5A
:101460001019019B489A02F04FFE0444002001909D
:1014700000BF002C0CDDFF2C0ADC0D222046641C72
:1014800002A90A54FF2C03DC0A222046641C0A54D9
:10149000002C03DDA1B202A802F0E2F800BFBEE713
:1014A000780000204D41494E00000000645D0008B6
:1014B0005B25735D5B25735D20000000704772B68D
:1014C00000BFFEE70146002291F82100022808D063
:1014D0000420886300BF002081F8200000BF0120A5
:1014E00070470868006820F00E000B6818600868F4
:1014F000006820F001000B68186091F8403001206E
:101500009840CB6B5860012081F8210000BF00207B
:1015100081F8200000BF1046E2E7000070B50446E5
:10152000002594F82100022803D00420A06301259F
:1015300048E02068006820F00E00216808602068FC
:10154000006820F00100216808601F492068884277
:1015500001D1012026E01C4914312068884201D1C4
:1015600010201FE0184928312068884201D18015D9
:1015700018E015493C312068884201D1801411E0FF
:10158000114950312068884202D14FF4803009E07F
:101590000D4964312068884202D14FF4801001E087
:1015A0004FF08070084908394860012084F8210014
:1015B00000BF002084F8200000BF606B10B12046FF
:1015C000616B8847284670BD0800024070B504462C
:1015D00000F0AEF906462546681C10B104480078B4
:1015E000054400BF00F0A4F9801BA842FAD370BDE7
:1015F000840000202DE9F8470346002294466EE15E
:101600004FF0010808FA02F4D1F8008008EA04005B
:10161000A0427DD1DFF8DCA2D1F80480A8EB0A0952
:10162000D0453AD014DCB8F1030F50D009DCB8F142
:10163000000F31D0B8F1010F1CD0B8F1020F49D121
:1016400020E0B8F1110F18D0B8F1120F42D11EE00E
:10165000B9F5881F25D006DCB9F5803F20D0B9F553
:10166000801F37D11AE0B9F5001F18D0B9F5041F53
:1016700030D117E0D1F80CC02DE0D1F80C8008F182
:10168000040C28E0D1F80C8008F1080C23E0D1F814
:101690000C8008F10C0C1EE000BF00BF00BF00BFB3
:1016A00000BF00BFD1F80880B8F1000F02D14FF0A1
:1016B000040C0BE0D1F80880B8F1010F03D14FF012
:1016C000080C1C6102E04FF0080C5C6103E04FF075
:1016D000000C00E000BF00BFFF2801D8984601E0E1
:1016E00003F104084646FF2802D84FEA820803E0C7
:1016F000A2F108084FEA88084746D6F800804FF064
:101700000F0909FA07F928EA09080CFA07F900E0B5
:1017100088E048EA0908C6F80080D1F8048008F09B
:101720008058B8F1805F7DD100BFDFF8CC81D8F858
:10173000188048F00108DFF8C091C9F81880C84641
:10174000D8F8188008F00108CDF8008000BF00BF6D
:101750004FEAB9384FEA920958F829504FEA82788F
:101760004FEA18794FF00F0808FA09F825EA08053A
:10177000DFF88881434502D14FF0000816E0DFF81A
:101780008081434502D14FF001080FE0DFF87481FA
:10179000434502D14FF0020808E0DFF86C81434571
:1017A00002D14FF0030801E04FF004084FEA8279BC
:1017B0004FEA197908FA09F848EA0505DFF84C817B
:1017C0004FEA920948F82950D1F8048008F48018AB
:1017D000B8F5801F0AD1DFF83881D8F8008048EAD0
:1017E0000008DFF82C91C9F8008009E0DFF82081BB
:1017F000D8F8008028EA0008DFF81491C9F80080C2
:10180000D1F8048008F40018B8F5001F10D1DFF8F3
:10181000008108F10408D8F8008048EA0008DFF8E1
:10182000F09000E05AE009F10409C9F800800DE0E9
:10183000DFF8DC8008F10408D8F8008028EA000806
:10184000DFF8CC9009F10409C9F80080D1F80480D0
:1018500008F40038B8F5003F0ED1DFF8B480A8F1E5
:101860000408D8F8008048EA0008DFF8A490A9F13D
:101870000409C9F800800DE0DFF89480A8F104089D
:10188000D8F8008028EA0008DFF88490A9F104095C
:10189000C9F80080D1F8048008F48038B8F5803F9A
:1018A0000ED1DFF86C80A8F10808D8F8008048EA6B
:1018B0000008DFF85C90A9F10809C9F800800DE084
:1018C000DFF84C80A8F10808D8F8008028EA000862
:1018D000DFF83C90A9F10809C9F80080521CD1F842
:1018E000008028FA02F8B8F1000F7FF489AEBDE855
:1018F000F8870000000011100010024000080140AD
:10190000000C01400010014000140140080001409B
:1019100008040140024693680B400BB1012000E02F
:10192000002070470AB1016101E00B0403617047B8
:1019300001480068704700007C00002003480068F0
:101940000349097808440149086070477C00002079
:101950008400002010B50848006840F010000649D7
:101960000860032000F0A8F80F2000F007F800F04E
:101970002BF8002010BD00000020024070B5044686
:101980000E4800784FF47A71B1FBF0F00C49096809
:10199000B1FBF0F5284600F09DFC08B1012070BDB8
:1019A000102C07D200222146501E00F047F80548AF
:1019B000046001E00120F2E70020F0E7840000204D
:1019C000880000208000002008B500BF1148806911
:1019D00040F001000F4988610846806900F001006D
:1019E000009000BF00BF00BF0846C06940F08050B3
:1019F000C8610846C06900F08050009000BF00BF79
:101A000000BF0549486820F0E06040F00070486081
:101A100000BF08BD0010024000000140014608461A
:101A2000002809DB00F01F0301229A4043099B00B4
:101A300003F1E023C3F8002100BF70472DE9F05FF8
:101A400080460D461646002702F078FB07463946C9
:101A50002A46334601F00700C0F1070ABAF1040F25
:101A600002D94FF0040A01E0C0F1070AD14600F1A3
:101A7000040ABAF1070F02D24FF0000A01E0A0F108
:101A8000030AD4464FF0010A0AFA09FAAAF1010A38
:101A90000AEA020A0AFA0CFA4FF0010B0BFA0CFBE5
:101AA000ABF1010B0BEA030B4AEA0B04214640465B
:101AB00002F04CFBBDE8F09F00BF00F00702064BB0
:101AC00019684FF6FF031940044B0B4343EA022108
:101AD000014B196000BF70470CED00E00000FA05F3
:101AE00070B504460D460CB9012070BD5A48006817
:101AF00000F00700A8420ED25748006820F0070007
:101B00002843554908600846006800F00700A842CD
:101B100001D00120E9E7207800F0020002281DD161
:101B2000207800F00400042805D14C48406840F4B7
:101B3000E0604A494860207800F00800082805D194
:101B40004648406840F46050444948604348406813
:101B500020F0F000A168084340494860207800F078
:101B6000010078B36068012806D13C48006800F4A1
:101B7000003090B90120B8E76068022806D13748E4
:101B8000006800F0007040B90120AEE733480068FB
:101B900000F0020008B90120A7E73048406820F0B3
:101BA0000300616808432D494860FFF7C1FE0646FF
:101BB00009E0FFF7BDFE801B41F28831884202D95F
:101BC000032092E707E02548406800F00C006168B8
:101BD000B0EB810FEDD12048006800F00700A8426B
:101BE0000ED91D48006820F0070028431A490860F4
:101BF0000846006800F00700A84201D0012074E701
:101C0000207800F00400042807D11448406820F42C
:101C1000E060E168084311494860207800F008005E
:101C2000082808D10D48406820F46050216940EA36
:101C3000C1000A49486000F03FF808494968C1F30B
:101C40000311074A515CC84006490860064800680D
:101C5000FFF794FE002048E70020024000100240F9
:101C60009E5D000888000020800000200148006878
:101C7000704700008800002000B5FFF7F7FF044917
:101C80004968C1F30221034A515CC84000BD00000D
:101C900000100240AE5D000800B5FFF7E7FF044901
:101CA0004968C1F3C221034A515CC84000BD00002D
:101CB00000100240AE5D000870B500210022002433
:101CC00000230020134D696801F00C05F5B1042DC7
:101CD00002D0082D19D101E00F4819E00F4DC1F3D2
:101CE0008346AB5D01F4803555B10A4D6D68C5F38F
:101CF00040450B4E725D084D5D43B5FBF2F402E0CA
:101D0000084D03FB05F4204602E000BF024800BF77
:101D100000BF70BD0010024000127A008C5D000808
:101D20009C5D000800093D00F8B504460CB901208F
:101D3000F8BD207800F00100002878D0F84840680D
:101D400000F00C0004280CD0F548406800F00C00AE
:101D5000082811D1F248406800F48030B0F5803F87
:101D60000AD1EF48006800F4003000285FD06068B6
:101D700000285CD10120DBE700BF6068B0F5803F40
:101D800006D1E748006840F48030E549086028E063
:101D9000606858B9E248006820F48030E049086083
:101DA0000846006820F4802008601AE06068B0F5FA
:101DB000A02F0BD1DA48006840F48020D849086091
:101DC0000846006840F4803008600AE0D4480068A3
:101DD00020F48030D24908600846006820F4802052
:101DE000086000BF606888B1FFF7A2FD054606E005
:101DF000FFF79EFD401B642801D9032098E7C848DF
:101E0000006800F400300028F2D010E0FFF790FDE9
:101E1000054606E0FFF78CFD401B642801D903202E
:101E200086E7BF48006800F400300028F2D120782F
:101E300000F00200022857D1B948406800F00C00B9
:101E400050B1B748406800F00C00082818D1B448D9
:101E5000406800F4803098B9B148006800F0020092
:101E600020B12069012801D0012061E7AC48006859
:101E700020F0F800616940EAC100A949086033E038
:101E80002069E8B10120A7490860FFF751FD054628
:101E900006E0FFF74DFD401B022801D9032047E76C
:101EA0009F48006800F002000028F2D09C480068BB
:101EB00020F0F800616940EAC1009949086013E028
:101EC000002098490860FFF733FD054606E0FFF75C
:101ED0002FFD401B022801D9032029E79048006804
:101EE00000F002000028F2D1207800F00800082855
:101EF0002DD1A069B8B101208B490860FFF718FD0A
:101F0000054606E0FFF714FD401B022801D9032017
:101F10000EE78348406A00F002000028F2D001205A
:101F200001F078FA13E000207F490860FFF700FD18
:101F3000054606E0FFF7FCFC401B022801D9032000
:101F4000F6E67748406A00F002000028F2D12078D7
:101F500000F00400042873D100277148C06900F024
:101F6000805070B900BF6E48C06940F080506C4925
:101F7000C8610846C06900F08050009000BF00BFF3
:101F800001276A48006800F48070B0B967480068AB
:101F900040F4807065490860FFF7CAFC054606E01A
:101FA000FFF7C6FC401B642801D90320C0E65F4848
:101FB000006800F480700028F2D000BFE0680128BB
:101FC00006D15748006A40F001005549086227E0F1
:101FD000E06858B95248006A20F001005049086290
:101FE0000846006A20F00400086219E0E06805284D
:101FF0000BD14B48006A40F004004949086208468A
:10200000006A40F0010008620AE04548006A20F0DA
:102010000100434908620846006A20F00400086293
:1020200000BFE068A0B1FFF783FC054609E0FFF7B9
:102030007FFC401B41F28831884202D9032077E6B9
:1020400022E03748006A00F002000028EFD012E0DA
:10205000FFF76EFC054608E0FFF76AFC401B41F203
:102060008831884201D9032062E62D48006A00F0D9
:1020700002000028F0D1012F05D12948C06920F0C5
:1020800080502749C86100BFE069C8B32448406850
:1020900000F00C00082860D0E069022848D1002038
:1020A00020490866FFF744FC054606E0FFF740FCC0
:1020B000401B022801D903203AE61948006800F0C5
:1020C00000700028F2D1206AB0F5803F07D1144893
:1020D000406820F40030A168084311494860D4E901
:1020E000080108430E49496821F4741108430C495A
:1020F000486001200B490866FFF71AFC054607E017
:102100003DE0FFF715FC401B022801D903200FE634
:102110000348006800F000700028F2D02FE00000B3
:102120000010024000004242800442420070004021
:10213000002014490866FFF7FBFB054606E0FFF7A1
:10214000F7FB401B022801D90320F1E50E48006887
:1021500000F000700028F2D111E0E069012800D100
:10216000E6E50948466806F48031206A814204D1D8
:1021700006F47011606A814201D00120D8E5002088
:10218000D6E50000000042420010024010B50446AF
:102190000CB9012010BD606A38B96068B0F5827F63
:1021A00000D105E00021E16102E0002121616161CF
:1021B0000021A16294F8510028B9002084F8500051
:1021C000204600F043F8022084F85100206800689F
:1021D00020F0400021680860A08800F48270218906
:1021E00001F404410843A18901F400610843217C02
:1021F00001F002010843217D01F001010843218B18
:1022000001F400710843217F01F0380108432021C7
:10221000095D01F080010843218D01F4005108435C
:10222000216808600421A06901EA10402168486023
:102230002068C06920F400602168C86100206065E2
:10224000012084F851000020A4E7000010B586B0FA
:102250000446002002900390049005901A492068DB
:1022600088422FD100BF1948C06940F48040174907
:10227000C8610846C06900F48040019000BF00BFFB
:1022800000BF0846806940F0080088610846806900
:1022900000F00800019000BF00BF4FF42040029002
:1022A000022003900320059002A90948FFF7A2F934
:1022B0004FF48040029000200390049002A904484B
:1022C000FFF798F906B010BD00380040001002403A
:1022D000000C014070B504462546681EB0F1807FB1
:1022E00001D301200FE0681E4FF0E02148610F216B
:1022F0004FF0FF3001F02AFF00204FF0E02188610D
:1023000007200861002070BD704770472DE9F84F25
:102310000446206805682068C668206847694FF051
:102320000009CA4605F00F09B9F1000F0AD105F0FE
:10233000200038B106F0200020B1204601F00AFD4F
:10234000BDE8F88FB9F1000F7BD007F0010018B994
:1023500006F49070002874D005F0010030B106F446
:10236000807018B1606C40F00100606405F00400FA
:1023700030B107F0010018B1606C40F002006064F9
:1023800005F0020030B107F0010018B1606C40F0B8
:102390000400606405F0080048B106F0200010B9A0
:1023A00007F0010018B1606C40F008006064606CD8
:1023B000002845D005F0200028B106F0200010B11B
:1023C000204601F0C7FC20684069C0F3801A606CA9
:1023D00000F0080010B9BAF1000F2CD0204601F02F
:1023E00073FC2068406900F0400000B300BF00BFEC
:1023F0002168143151E8001F21F040002168143198
:1024000041E80002002AF3D100BFE06B50B17748E9
:10241000E16B4863E06BFFF781F888B1E06B416BDB
:1024200088470DE02046FFF770FF09E009E02046ED
:10243000FFF76BFF04E02046FFF767FF00206064B2
:102440007EE7206B012877D105F01000002873D0BB
:1024500006F010000028FAD000BF0020009020688D
:102460000068009020684068009000BF00BF2068AE
:10247000406900F0400000285FD0E06B00684068D1
:102480001FFA80F8B8F1000F55D0A08D404552DDFD
:10249000A4F82E80E06B8069202843D000BF00BFE5
:1024A00021680C3151E8001F21F4807021680C3143
:1024B00041E80002002AF3D100BF00BF00BF21683D
:1024C000143151E8001F21F001002168143141E866
:1024D0000002002AF3D100BF00BF00BF2168143101
:1024E00051E8001F21F040002168143141E800024A
:1024F000002AF3D100BF202084F84200002020638E
:1025000000BF00BF21680C3151E8001F21F010000E
:1025100021680C3141E80002002AF3D100BFE06BD2
:10252000FEF7D0FF02206063A08DE28D801A81B299
:102530002046FFF7E9FE03E742E0A08DE18D401A57
:102540001FFA80F8E08DD0B3B8F1000F37D000BF8C
:1025500000BF21680C3151E8001F21F49070216800
:102560000C3141E80002002AF3D100BF00BF00BFD8
:102570002168143151E8001F21F001002168143155
:1025800041E80002002AF3D100BF202084F8420075
:102590000020206300BF00BF21680C3151E8001FFC
:1025A00021F0100021680C3141E80002002AF3D12B
:1025B00000BF0220606341462046FFF7A5FEBFE64C
:1025C00005F0800030B106F0800018B1204601F01F
:1025D000DDFCB5E605F0400030B106F0400018B172
:1025E000204601F0A7FBABE600BFA9E6B53C00081A
:1025F00010B504460CB9012010BDA06900B100E07F
:1026000000BF94F8410028B9002084F8400020461B
:1026100000F02AF8242084F841002068C06820F4E3
:1026200000502168C860204601F012FC2068006953
:1026300020F49040216808612068406920F02A0059
:10264000216848612068C06840F400502168C86073
:1026500000206064202084F8410084F842000020BB
:10266000606300BFC8E7000010B586B004460020D4
:10267000029003900490059059492068884237D110
:1026800000BF5848806940F4804056498861084638
:10269000806900F48040019000BF00BF00BF084681
:1026A000806940F0040088610846806900F00400F9
:1026B000019000BF00BF4815029002200390032044
:1026C000059002A94848FEF795FF4FF480600290FC
:1026D00000200390049002A94348FEF78BFF0022DC
:1026E00011462520FFF7AAF92520FFF797F975E095
:1026F0003E492068884236D100BF3A48C06940F45C
:1027000000303849C8610846C06900F400300190C3
:1027100000BF00BF00BF0846806940F00400886128
:102720000846806900F00400019000BF00BF04204B
:102730000290022003900320059002A92A48FEF788
:1027400059FF0820029000200390049002A9264817
:10275000FEF750FF002201212620FFF76FF9262007
:10276000FFF75CF93AE022492068884236D100BF81
:102770001C48C06940F480201A49C8610846C069F5
:1027800000F48020019000BF00BF00BF08468069B0
:1027900040F0080088610846806900F00800019058
:1027A00000BF00BF0815029002200390032005908F
:1027B00002A91048FEF71EFF4FF4006002900020AF
:1027C0000390049002A90B48FEF714FF0022022197
:1027D0002720FFF733F92720FFF720F906B010BDB7
:1027E0000038014000100240000801400044004051
:1027F00000480040000C014070B504460D461646E6
:1028000094F8420020280BD105B10EB9012070BD0B
:102810000020206332462946204601F097FBF6E768
:102820000220F4E770B5044616492068884208D1B2
:102830001548057802F064FE2946002000F06EFA83
:102840001FE01249206888420DD1FFF771F8054654
:1028500029460F480078FEF78FFA01220C490D48EF
:10286000FFF7CAFF0DE00C492068884209D10B48E8
:102870000178022000F052FA012208490848FFF7C7
:10288000BBFF70BD00380140AC0000200044004098
:1028900004000020A40100200048004005000020A2
:1028A000EC0100202DE9F84F04460E4617469946E4
:1028B0004FF0000A94F8410020284AD106B117B918
:1028C0000120BDE8F88F00206064212084F84100D9
:1028D000FFF72EF88246A784E784A068B0F5805FF2
:1028E00004D1206910B90025B04602E035464FF00A
:1028F00000081BE05346002280212046CDF80090BE
:1029000001F074FB08B10320DBE745B9B8F800001B
:10291000C0F308002168486008F1020803E0287845
:10292000216848606D1CE08C401EE084E08C00282B
:10293000E0D15346002240212046CDF8009001F01E
:1029400055FB08B10320BCE7202084F8410000209B
:10295000B7E70220B5E710B5034693F841002028F9
:1029600013D101B10AB9012010BD19629A84DA8429
:1029700000205864212083F841001868C06840F0A6
:1029800080001C68E0600020EEE70220ECE7000019
:1029900010B504460B492068884203D1002000F09E
:1029A000FBFA0DE008492068884202D100F0F6FEEB
:1029B00006E006492068884202D1022000F0ECFAC5
:1029C00010BD0000003801400044004000480040B5
:1029D00000BFFEE70021002009E0074A02EB0012D9
:1029E00092791AB1012282400A43D1B2401C0428D4
:1029F000F3DB084670470000100000200146042960
:102A000001DB00207047024800EB01108079F9E7F4
:102A10001000002070B5002512E0114800EB0514ED
:102A2000A1882068FEF776FF08B1012000E00020B1
:102A3000A071A07920720120E0710020E0606D1C7F
:102A4000042DEADB002007490860012006490870D0
:102A5000FFF7C0FF0446214604A000F0E1FD70BD71
:102A60001000002050000020540000205B494F5D02
:102A700020496E6974204F4B2C20696E697469611E
:102A80006C207374617465733A2030782530325845
:102A90000D0A00002DE9F041FEF74AFF07461C48E9
:102AA0000068381A0A2801D2BDE8F081184807608A
:102AB000002628E0174800EB0614A1882068FEF7DE
:102AC00029FF08B1012000E000200546207AA84235
:102AD00003D00020E071257214E0E079032803DAC6
:102AE000E079401CE0710DE0A079A8420AD0A57100
:102AF000E068401CE0600848007818B1F0B2294650
:102B000002F08CFF761C042ED4DB00BFCCE7000063
:102B100050000020100000205400002000B585B0B7
:102B20000020019002900390049000BF3C4880690F
:102B300040F010003A4988610846806900F01000B2
:102B4000009000BF00BF00BF0846806940F0200031
:102B500088610846806900F02000009000BF00BF37
:102B600000BF0846806940F004008861084680691B
:102B700000F00400009000BF00BF00BF084680695D
:102B800040F0080088610846806900F00800009065
:102B900000BF00BF012280212248FEF7C3FE0122B0
:102BA00005212148FEF7BEFE002241F208211E4801
:102BB000FEF7B8FE00224FF401411A48FEF7B2FEBC
:102BC00048F2801001900120029000200390022022
:102BD000049001A91348FEF70DFD41F20D2001906C
:102BE00001200290002003900220049001A90E48C9
:102BF000FEF700FD022001900020029001200390CA
:102C000001A90948FEF7F6FCF0200190002002908F
:102C1000039001A90448FEF7EDFC05B000BD0000DB
:102C20000010024000080140000C014010B50E48A1
:102C30000E4908604FF48270486000210B488160A3
:102C4000C160016141614FF4007181610021C16186
:102C50000162416281620A21C162FFF797FA08B1FD
:102C6000FEF72DFC10BD00000038004004010020DC
:102C700010B50B480B4908604FF41650486000210E
:102C800008488160C16001610C21416100218161BE
:102C9000C161FFF7ADFC08B1FEF711FC10BD0000EB
:102CA000003801405C01002010B50B480B4908605A
:102CB0004FF4E1304860002108488160C160016143
:102CC0000C21416100218161C161FFF791FC08B1D4
:102CD000FEF7F5FB10BD000000440040A4010020F9
:102CE00010B50B480B4908604FF41650486000219E
:102CF00008488160C16001610C214161002181614E
:102D0000C161FFF775FC08B1FEF7D9FB10BD0000EB
:102D100000480040EC01002000BFFEE770B505460A
:102D20000E46032D00DB70BD6B2068430E4901EB9E
:102D3000800494F8A80100B9F5E7314604F10800D1
:102D400002F02BFE40B9D4F8A401401CC4F8A40141
:102D500006A0616800F064FCD4F89C01401CC4F833
:102D60009C0100BFDFE700006C0600205B4D554171
:102D700052545D202573205258206F766572666C20
:102D80006F770D0A000000000146032901DB03A054
:102D90007047044850F82100FAE70000554E4B4EAA
:102DA0004F574E00805D00080146032901DB0020DB
:102DB000704772B66B204843034B03EB8000B0F8BA
:102DC0008C2062B61046F3E76C060020014603290A
:102DD00001DB0020704772B66B204843054B03EBC4
:102DE0008000B0F89401C0F5807082B262B61046DF
:102DF000F0E700006C06002070B5002520E06B2095
:102E00006843134901EB8004124850F82500206004
:102E1000114850F82500606004F1080002F0B5FD8B
:102E200004F1900002F037FF002004F5CE7404F89E
:102E3000020C20606060A06001202073681CC5B295
:102E4000032DDCDB032105A000F0EAFB70BD0000D0
:102E50006C060020745D0008805D00085B4D5541E4
:102E600052545D20496E6974204F4B2C20256420FC
:102E7000706F72747320636F6E66696775726564D4
:102E80000D0A000010B502460B46032A00DA0BB902
:102E9000002010BD6B205043104C04EB800000F16B
:102EA000080172B6B1F8840010B962B60020F0E7EC
:102EB000B1F88200085C187031F8824F601CC417AA
:102EC00000EB5464E411A0EBC4140C804888401E4D
:102ED0004880823962B60120DBE700006C060020E2
:102EE0002DE9F04105460F469046032D03DA17B150
:102EF000B8F1000F01D1BDE8F081012D04D14146A8
:102F0000384600F0ADFBF6E76B2068430C4901EB57
:102F1000800494F8A80100B9EDE74246394604F16F
:102F2000900002F0C3FE0646002E07DDD4F8A00193
:102F30003044C4F8A001284602F070FE00BFDAE772
:102F40006C06002070B505460C4604B970BD2046DD
:102F5000FDF72BF986B2324621462846FFF7C0FF1F
:102F600000BFF3E770B5002411E06B20604309490E
:102F700001EB800595F8A80100B906E0012C00D10D
:102F800003E0204602F04AFE00BF601CC4B2032CDE
:102F9000EBDB70BD6C060020F8B50546032D00DBA9
:102FA000F8BD012D02D100F0F9FBF9E76B20684371
:102FB000164901EB800606F19004002772B6002046
:102FC00084F80601B4F80401002816DDB4F8020103
:102FD000205C009004F581742188481CC11700EB27
:102FE00011610912A0EB012121806088401E6080E0
:102FF00001202071A4F58174012762B627B1012256
:1030000069463068FFF7A7FC00BFC9E76C060020DF
:1030100000BFFEE710B50020FFF7D8FE002806DD50
:103020000448B0F81A02002801DD012010BD00207C
:10303000FCE70000700B002010B54FF40C711F4826
:10304000FDF7A8F800201BE0002100EB400202EB96
:1030500080121A4B03EB420282F8841000EB40020C
:1030600002EB801203EB4202A2F8801000EB400258
:1030700002EB801203EB4202A2F88210411CC8B29C
:103080000428E1DB00200D4981F8180281F81902BB
:10309000A1F81A02C1F81C0200210848C0F8201249
:1030A000C0F82412C0F828120120044981F82C022B
:1030B000410203A000F0B4FA10BD0000700B002024
:1030C0005B5054585D20506173737468726F7567FC
:1030D0006820656E67696E6520696E697469616CE8
:1030E000697A65642C206275666665722073697AF8
:1030F000653A2025642062797465730D0A0000002A
:103100002DE9F04781460F46B9F1000F00D017B9FD
:103110000020BDE8F087374C0026B04656E094F812
:103120001812481CC11700EB91718910A0EB8101A6
:1031300001F0FF0A94F81902504510D1B4F81A02B0
:1031400000280CDD4FF409700059401C4FF4097140
:1031500008513A46414628A000F062FA38E094F857
:10316000180200EB400101EB801004EB400595F8DC
:10317000840018B1B5F88000802813DB95F884002E
:1031800048B184F818A294F8180200EB400101EB52
:10319000801004EB4005002025F8800F6880012096
:1031A0002871803D19F8081035F8802F2888401CB8
:1031B00025F88009A954B4F81A02401CA4F81A0290
:1031C000701C86B208F101001FFA80F8B845A6DB32
:1031D00000BF002E0CDD4FF408700059401C4FF466
:1031E00008710851B4F81A2231460DA000F018FAFF
:1031F00030468EE7700B00205B5054585D204275BE
:1032000066666572206F766572666C6F7720617492
:1032100020627974652025642F25640D0A00000062
:103220005B5054585D205075736865642025642098
:10323000627974657320746F206275666665722C9E
:103240002070656E64696E673A2025640D0A00007F
:103250002DE9F04107462C4C94F82C0210B90020BF
:10326000BDE8F08194F81812481CC11700EB917169
:103270008910A0EB8101CEB294F81902B04211D1AD
:10328000B4F81A0200280DDD4FF409700059401CF3
:103290004FF409710851084601591CA000F0C0F90B
:1032A0000020DDE794F8180200EB400101EB8010EC
:1032B00004EB400595F8840018B1B5F8800080282B
:1032C00013DB95F8840048B184F8186294F818026A
:1032D00000EB400101EB801004EB4005002025F8D5
:1032E000800F688001202871803D35F8801F288874
:1032F000401C25F880096F54B4F81A02401CA4F849
:103300001A020120ACE70000700B00205B505458FB
:103310005D204275666665722066756C6C2C206F48
:10332000766572666C6F7720636F756E743A2025D0
:10333000640D0A0038B52B4C94F82C0200B938BD46
:10334000B4F81A0200B9FAE7FFF764FE38B94FF48F
:103350000A700059401C4FF40A710851EFE794F8C5
:10336000190200EB400101EB801004EB400595F8D9
:10337000840028B1B5F88200B5F88010884211DBCE
:1033800095F8840010B1002085F8840094F8191293
:10339000481CC11700EB91718910A0EB810184F8E2
:1033A0001912CCE735F8821F2888401C25F88209BD
:1033B000685C0090012269460020FFF791FDB4F897
:1033C0001A02401EA4F81A02D4F81C02401CC4F8C9
:1033D0001C02B4F81A229DF8001003A000F020F996
:1033E00000BFACE7700B00205B5054585D20536564
:1033F0006E742062797465203078253032582C2024
:1034000070656E64696E673A2025640D0A000000DD
:103410007047000008B508490968C9084FF47A7276
:10342000B1FBF2F14143009100BF00BF00994A1E79
:1034300000920029F9D108BD8800002010B50022B3
:103440004FF400410548FEF76DFA0020044908706A
:103450000449086004A000F0E3F810BD0008014032
:103460005C000020600000205B52454C41595D200B
:10347000496E6974204F4B2C2073746174653D4F05
:1034800046460D0A0000000070B50446FEF750FAEB
:10349000054615480068281A642803D213A000F0D6
:1034A000BFF870BD1A480078A04208D10CB119A02D
:1034B00000E019A0014619A000F0B2F8F1E7224699
:1034C0004FF400411D48FEF72DFA114804700648DC
:1034D00005600CB10FA000E00FA0014618A000F09D
:1034E0009FF800BFDDE70000600000205B52454C04
:1034F00041595D20546F67676C6520746F6F20665B
:103500006173742C2069676E6F7265640D0A000028
:103510005C0000204F4E00004F4646005B52454C79
:1035200041595D20537461746520756E6368616EE6
:103530006765643A2025730D0A0000000008014009
:103540005B52454C41595D2052656C6179202D3E9E
:103550002025730D0A000000704710B502F02CFB07
:10356000FEF7ECF910BD00B58FB0282105A8FCF7D7
:1035700011FE14216846FCF70DFE012005900004A1
:103580000690002007900120099002200C90C103B2
:103590000D914FF4E0110E9105A8FEF7C5FB08B19F
:1035A000FDF78DFF0F200090022001900020029077
:1035B0004FF4806003900020049002216846FEF7DB
:1035C0008FFA08B1FDF77BFF0FB000BD7047000018
:1035D00010B500200849A1F80001A1F80201A1F8E6
:1035E000040181F80601A1F808014FF4807103A0DD
:1035F00000F016F810BD0000940200205B55415207
:1036000054325D20496E6974204F4B2C20627566E0
:103610006665722073697A653A2025640D0A000098
:103620000FB410B5A2B0249818B922B010BC5DF840
:1036300014FB25A80190802102A8019B249A00F088
:1036400063FD044600200190002C06DB802C00DB8B
:103650007F24A1B202A800F003F800BFE5E7000054
:10366000F8B504460D4605B104B9F8BD002600279B
:1036700072B6002029E02549B1F80411FF2907DDC1
:103680002249B1F80811491C204AA2F808111EE08D
:10369000215C1E4AB2F800211C4B99541A46B2F81C
:1036A0000021511CCA1701EB12621212A1EB022277
:1036B000A3F800211946B1F80411491C1A46A2F8D2
:1036C0000411711C8EB2411C88B2A842D3DB00BF2A
:1036D000002E08DD0D4890F8060120B901200B49A5
:1036E00081F80601012762B66FB172B60748B0F8DB
:1036F00002010649085C009062B60122694604484E
:10370000FFF729F900BF00BFAFE7000094020020D7
:10371000A401002070B5044604B970BD2046FCF732
:1037200044FD85B229462046FFF79AFF00BFF4E723
:1037300038B572B6174890F8060118B91548B0F8B0
:10374000040108B962B638BD1248B0F8024101461A
:10375000B1F80211481CC11700EB11610912A0EB6E
:1037600001210C4AA2F802111046B0F80401401ED3
:103770001146A1F80401012081F806010846005D08
:10378000009062B6012269460348FFF7E4F800BFE3
:10379000D9E7000094020020A401002038B50025DC
:1037A00072B60020164981F806010846B0F80401F7
:1037B00000281CDD0846B0F80241B1F80211481C8F
:1037C000C11700EB11610912A0EB01210C4AA2F80C
:1037D00002111046B0F80401401E1146A1F8040180
:1037E000012081F806010846005D0090012562B6BF
:1037F00025B1012269460348FFF7ADF838BD000046
:1038000094020020A401002070B50546134C2078D6
:1038100001280FD1B4F88C0000280BDDA068281A0D
:10382000322807D30420207032210DA0FFF7F8FEC4
:10383000012070BD207802280DD16068281AC828A0
:1038400009D300202070A4F88C00C82110A0FFF735
:10385000E7FE0120EDE70020EBE70000A00D0020CF
:103860005B50524F544F5D205343414E2074696D5D
:10387000656F757420E2869220504153535448522C
:103880004F55474820282564206D73290D0A0000F4
:103890005B50524F544F5D20434D445F4D4F444564
:1038A0002074696D656F757420E2869220494E49D7
:1038B0005420282564206D73290D0A0070B5054633
:1038C0000E46484C207880B1207801280DD0207811
:1038D00002280AD02078042807D000202070A4F8FD
:1038E0008C00217840A0FFF79BFE21782A464CA04F
:1038F000FFF796FE207830B101281DD002284CD069
:10390000042867D15FE06660242D09D10220207071
:103910000020A4F88C004DA0FFF782FE012070BDAE
:1039200001202070A6602573A4F88C00294651A0C0
:10393000FFF776FE0020F2E76660242D13D1B4F87D
:103940008C00002808DD04202070B4F88C1053A0EF
:10395000FFF766FE0220E2E7022020705CA0FFF77E
:103960005FFE0120DBE70A2D08D104202070B4F8A7
:103970008C1064A0FFF754FE0220D0E7B4F88C004E
:10398000802808D234F88C1F2088401C24F88C0929
:1039900004F10C0045540020C1E766600A2D08D1EF
:1039A00000202070A4F88C0063A0FFF739FE0120EE
:1039B000B5E70D2D01D10120B1E7294668A0FFF739
:1039C0002FFE0120ABE7294670A0FFF729FE6660B5
:1039D0000220A4E70020207078A0FFF721FE00203D
:1039E0009DE70000A00D00205B50524F544F5D201A
:1039F00050726F746F636F6C2073746174652069AB
:103A00006E76616C696428307825303258292C2014
:103A1000726573657420746F20494E49540D0A0015
:103A20005B50524F544F5D20466565644279746522
:103A30002073746174653D25642C20627974653D42
:103A40003078253032580D0A000000005B50524F8C
:103A5000544F5D20494E495420E2869220434D4404
:103A60005F4D4F44452028676F7420272427290D78
:103A70000A0000005B50524F544F5D20494E49549C
:103A800020E28692205343414E2028627974653AA1
:103A900020307825303258290D0A00005B50524FF3
:103AA000544F5D205343414E20E2869220504153B3
:103AB000535448524F5547482028676F7420272495
:103AC000272C202564206279746573290D0A000073
:103AD0005B50524F544F5D205343414E20E286923B
:103AE00020434D445F4D4F44452028656D707479E7
:103AF000207363616E2C20676F7420272427290DA3
:103B00000A0000005B50524F544F5D205343414E1A
:103B100020E2869220504153535448524F55474813
:103B20002028676F7420275C6E272C202564206274
:103B300079746573290D0A005B50524F544F5D2014
:103B4000434D445F4D4F444520E2869220494E4903
:103B5000542028676F74205C6E290D0A0000000055
:103B60005B50524F544F5D20434D445F4D4F444591
:103B700020E2869220434D442028627974653A20E1
:103B8000307825303258290D0A0000005B50524F22
:103B9000544F5D20504153535448524F554748208D
:103BA000E28692205054582028627974653A203079
:103BB0007825303258290D0A000000005B50524F22
:103BC000544F5D20556E6B6E6F776E207374617409
:103BD000652C20726573657420746F20494E4954BA
:103BE0000D0A000070B506460D46104C20780428DA
:103BF00019D1B4F88C00002815DD56B14DB1B4F8D8
:103C00008C2004F10C013046FCF7ABFAB4F88C00C0
:103C100028800020A4F88C002070298804A0FFF7D9
:103C2000FFFC012070BD0020FCE70000A00D00207B
:103C30005B50524F544F5D204765745061737374ED
:103C400068726F756768446174613A202564206208
:103C5000797465732C206261636B20746F20494E08
:103C600049540D0A0000000010B594210448FCF7E7
:103C700091FA00200249087002A0FFF7D1FC10BDA4
:103C8000A00D00205B50524F544F5D2050726F7456
:103C90006F636F6C206469736372696D696E6174C0
:103CA0006F7220696E697469616C697A65640D0A66
:103CB0000000000070B505466C6A0020E085E084D5
:103CC0002046FEF722FB70BD00BF00BF02680C3229
:103CD00052E8002F22F4907102680C3242E800137F
:103CE000002BF3D100BF00BF00BF0268143252E8BE
:103CF000002F22F001010268143242E80013002B69
:103D0000F3D100BF016B01290ED100BF00BF0268D3
:103D10000C3252E8002F22F0100102680C3242E807
:103D20000013002BF3D100BF202180F842100021A6
:103D30000163704710B504462068C06820F0400059
:103D40002168C860202084F841002046FEF720FE4C
:103D5000002010BDF8B5044694F84200222875D121
:103D6000A068B0F5805F0CD1206950B90025A66A23
:103D700020684068C0F308003080A06A801CA06200
:103D800015E0A56A0026A068B0F5805F03D0A068A2
:103D900028B9206918B920684068287004E02068B4
:103DA000406800F07F002870A06A401CA062E08D8F
:103DB000401E80B2E085002846D12068C06820F00F
:103DC00020002168C8602068C06820F480702168E5
:103DD000C8602068406920F0010021684861202007
:103DE00084F8420000206063206B012826D1002067
:103DF000206300BF00BF21680C3151E8001F21F093
:103E0000100021680C3141E80002002AF3D100BF04
:103E10002068006800F0100010280AD100BF0020C0
:103E2000009020680068009020684068009000BF03
:103E300000BFA18D2046FEF767FA02E02046FEF79C
:103E4000F1FC0020F8BD01E00020FBE70220F9E7CB
:103E500070B504462168096921F44051E2681143B4
:103E6000226811612269A1681143626941EA020571
:103E70002168C96841F20C62914329432268D160EC
:103E80002168496921F44071A26911432268516196
:103E90002D4A2168914202D1FDF7FEFE01E0FDF7B7
:103EA000EBFE00EBC00101EB001162689200B1FB78
:103EB000F2F100EBC00202EB001263689B00B2FB60
:103EC000F3F26423B2FBF3F202EBC20303EB021240
:103ED000A1EB8201322202EB01116422B1FBF2F16B
:103EE00001F0F00100EBC00202EB001263689B00DE
:103EF000B2FBF3F26423B2FBF3F201EB021200EB2C
:103F0000C00101EB001163689B00B1FBF3F100EB12
:103F1000C00303EB00136668B600B3FBF6F3642638
:103F2000B3FBF6F303EBC30606EB0313A1EB83012C
:103F3000322303EB01116423B1FBF3F101F00F0114
:103F400011442268916070BD0038014010B50346ED
:103F500099629A85DA8500205864222083F842000D
:103F6000186928B11868C06840F480701C68E06067
:103F70001868406940F001001C6860611868C068FA
:103F800040F020001C68E060002010BD014691F860
:103F90004100212828D18868B0F5805F0BD10869DD
:103FA00048B90A6A1088C0F308000B685860086AAC
:103FB000801C086205E00B6A581C086218780B68C0
:103FC0005860C88C401E80B2C88458B90868C06860
:103FD00020F080000B68D8600868C06840F040009E
:103FE0000B68D860002070470220FCE72DE9F04103
:103FF00004460D4617469846069E34E0701C88B36A
:104000002EB1FDF795FCA0EB0800B0422BD900BF04
:1040100000BF21680C3151E8001F21F4D0702168E5
:104020000C3141E80002002AF3D100BF00BF00BFFD
:104030002168143151E8001F21F00100216814317A
:1040400041E80002002AF3D100BF202084F841009B
:1040500084F8420000BF002084F8400000BF032025
:10406000BDE8F081FFE7206800682840A84201D140
:10407000012000E00020B842C0D00020F0E700009E
:1040800010B50248FEF742F910BD00005C010020A7
:1040900010B50248FEF73AF910BD0000A401002057
:1040A00010B50248FEF732F910BD0000EC01002007
:1040B00000BFFEE70FB4054B10B503A9044A0298F0
:1040C00000F02EF910BC5DF814FB0000FD4B000859
:1040D000B80000200FB47CB50C0009AD01D0611E02
:1040E00000E00021CDE90001064B6A462946089808
:1040F00000F016F9002C02D0009A002111707CBC4F
:104100005DF814FB274A00087CB50C001D461646D6
:10411000014601D0601E00E00020CDE90010064BF2
:104120006A462946304600F0FBF8002C02D0009A7F
:10413000002111707CBD0000274A00080248006879
:10414000C0F30220704700000CED00E010B500281D
:1041500004DB0A07130E054A135406E00A07140E7F
:10416000034A00F00F031B1FD45410BD00E400E00D
:1041700018ED00E000487047BC00002002E008C8CD
:10418000121F08C1002AFAD170477047002001E0D1
:1041900001C1121F002AFBD1704700002DE9FF5F0B
:1041A00082B00021DDE90430020DDDF840B00343A8
:1041B00018D044F61050A2F2FF3242431514119861
:1041C00001281FD0A5EB0B00401C5FEA000A4FF04E
:1041D00000064E4FDFF83891B046504615D5CAF16B
:1041E000000413E0119801244AA3012801D16FEAC9
:1041F0000B010298119AC0E90031C0E9024206B0F1
:10420000BDE8F09FCBF10000DFE704460021404A03
:10421000491842EB0450CDE9001012E0E00707D046
:1042200032463B4640464946FCF71BFA80468946E3
:1042300032463B4610461946FCF713FA06460F462F
:104240006410002CEAD1DDE90401DDE90023BAF1B4
:10425000000F06DAFCF705FA42464B46FCF701FA76
:1042600005E0FCF770FA42464B46FCF76CFA044650
:104270000E460022284BFCF7EDFA03D84FF0FF3032
:10428000014607E00022254B20463146FCF742F963
:10429000FCF7C8FA102409E0002C0ADB0A220023EC
:1042A000FCF78DF8039B30321A55641E50EA010268
:1042B000F2D1641C039AC4F111031444119A012A27
:1042C00003D0012208430DD10AE0084304D00020A6
:1042D0004FF0110B119072E7A3EB0B056D1E0DE073
:1042E0005B4504DD4FF0000205F1010504E003DA4F
:1042F0004FF00002A5F10105002AECD002981199B7
:10430000C0E90231C0E9004579E70000000014402F
:104310000000F03F300000000000F0430000E03FEC
:104320002DE9FF4F95B09A46884606460025EEE1F6
:10433000252877D100242746F94A0121039400E07B
:10434000044316F8013F203B01FA03F01042F7D175
:1043500030782A2811D06FF02F033078A0F1300286
:10436000092A16D8039A44F0020402EB820203EBF6
:1043700042021044761C0390EFE758F8042B039296
:10438000002A03DA504244F40054039044F002043B
:10439000761C30782E2816D116F8010F44F004044C
:1043A0002A280DD06FF02F023078A0F13003092BAE
:1043B00009D807EB870302EB4303C718761CF3E722
:1043C00058F8047B761C30786C280FD006DC4C281B
:1043D00017D068280DD06A2814D104E0742810D0B2
:1043E0007A280FD10DE044F400140AE044F480145C
:1043F00001E044F440147278824202D104F5801442
:10440000761C761C307866280BD013DC582877D0C1
:1044100009DC002875D04528F6D04628F4D0472876
:104420001AD193E118E0632835D0642879D0652843
:1044300012D18BE1702873D008DC6728F1D069288D
:104440006FD06E280DD06F2806D1ACE073282CD029
:10445000752874D0782853D05246179990476D1C10
:1044600054E1C4F30250022809D003280DD0D8F833
:10447000001004280DD00D6008F1040846E1D8F8BA
:104480000010EA17C1E90052F6E7D8F800100D80D5
:10449000F2E70D70F0E718F8041B8DF8001000200B
:1044A0008DF80100EB46012003E058F804BB4FF003
:1044B000FF3061074FF0000102D40DE009F1010166
:1044C0008946B9420FDA8145F8DB1BF8091000294B
:1044D000F4D108E009F1010189468142FADB1BF8B9
:1044E00009100029F6D103985346A0EB090721468D
:1044F0003846179A00F080FA284400EB090507E0D7
:1045000044E008E10DE01BF8010B52461799904773
:10451000B9F10109F7D2534621463846179AF2E01D
:1045200039E00A21C4F302524FF0000B0091022A35
:1045300006D058F8040BC117032A09D00AE023E07B
:1045400008F1070020F00702F2E80201904605E0BA
:1045500000B2C117042A01D140B2C117002906DAFE
:104560000A460021404261EB02012D2202E02205B1
:1045700004D52B228DF80420012203E0E20701D0AC
:104580002022F7E7914657E00A2100E010214FF082
:10459000000B00910BE010214FF0000B44F00404DD
:1045A0000827009103E008204FF0000B0090C4F3AF
:1045B0000252022A05D058F8040B0021032A08D021
:1045C00008E008F1070020F00702F2E80201904637
:1045D00003E080B2042A00D1C0B24FF000092207E4
:1045E0002AD53278702A07D0DDF800C08CF0100C84
:1045F0005CEA0B0C05D00EE040228DF8042001226D
:1046000008E050EA010306D030238DF804308DF81D
:10461000052002229146009B83F0080353EA0B0316
:104620000AD150EA010201D1620705D530228DF886
:1046300004204FF001097F1E3278582A04D039A295
:104640000C920CAA02920BE03BA2F9E75B46009A9F
:10465000FBF7B5FE0C9B9B5C029A521E02921370F4
:1046600050EA0102F2D1029804A9081A00F1200BC5
:10467000600702D524F4803400E001275F4502DDA5
:10468000A7EB0B0000E0002000EB0B01009003986B
:104690004944401A0390E00306D453462146179A32
:1046A000039800F0A9F90544002706E001A8524646
:1046B000C05D179990476D1C7F1C4F45F6DBE003EA
:1046C0000CD553462146179A039800F095F90544F6
:1046D00004E030205246179990476D1C0099481EFF
:1046E00000900029F5DC08E0029802995246007813
:1046F000491C0291179990476D1CBBF10001ABF169
:10470000010BF1DC5BE100F065F90544761C3078C3
:1047100000287FF40DAE19B02846BDE8F08F0000E8
:104720000928010030313233343536373839616287
:10473000636465660000000030313233343536374B
:10474000383941424344454600000000600700D428
:10475000062708F1070020F00700F0E80223804652
:1047600003F0004C5FEA0C0001D097A009E020059F
:1047700001D596A005E0E00701D095A001E0AFF2D9
:104780004C001390307823F0004365280CD006DCF1
:10479000452809D046281DD047287FD13BE0662810
:1047A00018D067287AD136E00021112F01DB1120C3
:1047B00000E0781CCDE9000104A90CA8FFF7EEFC8D
:1047C000DDE90D010C9A4FF0000B07F10109109281
:1047D00000914EE04FF000400097CDE9011004A990
:1047E0000CA8FFF7DBFCDDE90D020C9B0F994FF0E5
:1047F000000B91461093009211B9791C00EB01094E
:10480000B7EB090003D4C0F1FF3B07F10109A9EBA5
:104810000700019042E0012F00DA01270021112F4B
:1048200001DD112000E03846CDE9000104A90CA803
:10483000FFF7B4FCDDE90D010C9A00914FF0000B7D
:10484000B946109221070FD4009A4A4503DA9146DF
:1048500001E0A9F10109B9F1010F05DD109AA9F1F3
:104860000101515C3029F4D0B84202DA10F1040F92
:1048700003DA0121CDE9011010E0002803DC8344B4
:10488000A9EB000102E0411C494500DD8946A0EB8F
:104890000B00401C01904FF000400290200705D40F
:1048A0000198484502DB4FF0FF30019000208DF861
:1048B0004B0002980DF14B07B0F1004F25D00220BC
:1048C0000C902B200D90029800280CDA40420290A8
:1048D0002D200D9007E00A210298FBF75AFD303198
:1048E000029007F8011D0C99481E0C900029F2DC7B
:1048F00002980028EFD1791E0D980870307800F0EA
:10490000200040F0450007F8020D11A8C01BC01D93
:1049100002901398007800B1012000EB0901019882
:1049200001EBE071029801440398401A401E039085
:10493000E00306D453462146179A039800F05CF82A
:1049400005441398007818B15246179990476D1C8A
:10495000E00323D553462146179A039800F04CF8FC
:1049600005441BE0BBF1000F07DB0098584504DD50
:104970001098179910F80B0001E017993020524653
:10498000904701980BF1010B401E05F101050190C4
:1049900004D12E205246179990476D1CB9F10001A1
:1049A000A9F10109DEDC05E017F8010B5246179961
:1049B00090476D1C0299481E02900029F4DC534672
:1049C0002146179A03989EE62D0000002B00000058
:1049D000200000002DE9F041044600251E46174640
:1049E000880404D405E039462020B0476D1C641EBD
:1049F000F9D52846BDE8F0812DE9F04104460025AF
:104A00001E469046C80301D5302700E020278804C1
:104A100004D505E041463846B0476D1C641EF9D503
:104A20002846BDE8F0814A68002A06D00A68531C6F
:104A30000B6010704868401E4860704770B50446AF
:104A40000D460C4830F8140080280CDA094830F87C
:104A5000141030F81400401C064A22F814000648CE
:104A600000EBC4104554FCF763FF044941F82400EF
:104A700070BD000072000020D0030020500500200F
:104A800010B502460023002003E0145C6340441C80
:104A9000E0B28842F9DB184610BD10B5024600238B
:104AA000002003E0145C6340441CE0B28842F9DB60
:104AB000184610BDF8B505460C461448006878B194
:104AC0002046FBF772FB86B23246214628460F4B42
:104AD0001B6898470E480068401C0D49086008E0B4
:104AE00021462846FEF72EFA09480068401C08496E
:104AF00008602846FEF748F90646334605A208A195
:104B000001200094FCF782FCF8BD00006400002046
:104B10006C00002054585B25735D3A20257300001B
:104B2000524F5554455200007CB50446274830F892
:104B3000140000B97CBD2046FEF726F9054629463B
:104B400023A0FEF76DFD002531E0264800EBC410E0
:104B5000405D01909DF80400202808DB9DF80400CA
:104B60007F2804DA012101A8FEF77AFD1DE09DF8F7
:104B700004000D2804D102211BA0FEF771FD14E0F2
:104B80009DF804000A2804D1022118A0FEF768FD50
:104B90000BE09DF8043016A204216846FFF79AFA4C
:104BA00004216846FEF75CFD00BF681C85B207481B
:104BB00030F81400A842C8DC0FA0FEF7ABFD0020BF
:104BC000024921F8140000BFB4E700007200002081
:104BD0005B524F555445525D2025732052583A2060
:104BE00022000000D00300205C7200005C6E000018
:104BF0005C78253032580000220D0A0013B50C46AF
:104C000001216846FEF72CFD00981CBD10B500225E
:104C100008210248FCF786FE10BD0000000C014090
:104C200010B5012208210248FCF77CFE10BD0000EF
:104C3000000C014010B500224FF400710148FCF750
:104C400071FE10BD000C014010B501225102024856
:104C5000FCF768FE10BD0000000C01400146302941
:104C600005DB392903DCA1F13000C0B270474129CE
:104C700005DB462903DCA1F13700C0B2F6E7612964
:104C800005DB662903DCA1F15700C0B2EEE7002086
:104C9000ECE770B505460C462046FFF7DFFF0646F9
:104CA0002846FFF7DBFF46EA0010C0B270BD0000E7
:104CB0000B48007800B17047002009E0002100EBAC
:104CC0000012084B995400EB00121A441174401C56
:104CD0001028F3DB01200249087000BFEBE7000059
:104CE000790000205C05002070B505460DB12878DC
:104CF00008B9012070BDFFF7DBFF002414E004EBCE
:104D000004100B49085C70B104EB0411084A8818C0
:104D10000F222946FBF75EFA28B904EB0410044978
:104D20000844007CE6E7641C102CE8DB0120E1E786
:104D30005C050020014609B1087808B901207047D8
:104D40000020FCE710B504462046FFF7F3FF08B14A
:104D5000002010BD09E0FBF7F7F900682178405CFE
:104D6000202801D00020F4E7641C20780028F2D12C
:104D70000120EEE710B50446FBF7E6F90068005D98
:104D800000F0100028B9FBF7DFF90068005D20286B
:104D900001D1012010BD0020FCE710B50446FBF74F
:104DA000D3F90068005D00F03E0038B12A2C05D030
:104DB0000D2C03D00A2C01D0012010BD0020FCE7EF
:104DC000FCF7C8FDFEF7CFFBFDF7A8FEFDF750FF8F
:104DD000FDF72CFFFDF768FFFDF782FFFEF7F8FBFC
:104DE000FDF718FEFCF778F9FEF728FBFEF704F84C
:104DF000FCF7A6F9FCF7EAFA012220492048FDF762
:104E0000FBFC01221F492048FDF7F6FC002000F0C2
:104E1000A9FB01221D491E48FDF7EEFC002000F011
:104E200005FD4FF47A710A2000F026FD002000F005
:104E3000C9FB00F017FC17A0FFF73CF921A0FFF712
:104E400039F9294800682949B0FBF1F4214628A026
:104E5000FFF730F92CA0FFF72DF90DE0FEF768FC05
:104E6000FDF718FEFCF75AF9FEF77CF8FCF7D8F9C5
:104E700000F018FD00F006FCF0E700000400002040
:104E8000A401002005000020EC010020AC0000205F
:104E90005C0100200D0A3D3D3D3D3D3D3D3D3D3D1C
:104EA0003D3D3D3D3D3D3D3D3D3D3D3D3D3D3D3D32
:104EB0003D3D3D3D3D3D3D3D3D3D3D3D3D3D0D0A85
:104EC000000000004533322D3433335442482D5313
:104ED00043204170706C69636174696F6E20537414
:104EE00061727465640D0A008800002040420F0062
:104EF00053797374656D20436C6F636B3A2025643E
:104F0000204D487A0D0A00003D3D3D3D3D3D3D3D73
:104F10003D3D3D3D3D3D3D3D3D3D3D3D3D3D3D3DC1
:104F20003D3D3D3D3D3D3D3D3D3D3D3D3D3D3D3DB1
:104F30000D0A000070B58CB0044694F84C0008B11E
:104F400060A200E061A294F8490094F8481004F1CE
:104F50002803CDE90102009104F1080221465CA07A
:104F6000FEF75EFB65A12046FBF726F9002835D148
:104F700004F10800FFF7E6FE38B961A000F0B2FDC9
:104F800061A0FEF74DFB0CB070BD04F10800FBF70B
:104F9000F3F905460DB1012D18D10DB1012100E045
:104FA00000210846FEF770FA2B4661A2202104A8D2
:104FB000FFF790F804A800F0CBFD0DB15EA000E073
:104FC0005EA001465EA0FEF72BFB06E04CA000F0C1
:104FD00089FD29465FA0FEF723FB71E066A120460C
:104FE000FBF7EAF8002858D104F10800FFF7A2FE09
:104FF00028B962A104F10800FBF7DEF8D0B9FDF78B
:10500000E9FC0546C5F3C000C5F38001C5F34002C5
:1050100005F00103CDE90021029059A2202104A846
:10502000FFF758F804A800F093FD294657A0FEF7B3
:10503000F7FA45E004F10800FFF784FE002825D0C8
:1050400004F10800FBF798F90546012D16DB042D45
:1050500014DC691EC8B2FDF7D1FC06462B4653A2EC
:10506000202104A80096FFF735F804A800F070FD91
:105070003246294650A0FEF7D3FA06E020A000F001
:1050800031FD294651A0FEF7CBFA19E01CA000F033
:1050900029FD56A0FEF7C4FA12E05EA12046FBF7F8
:1050A0008BF830B95BA000F053FD5CA0FEF7B8FAB6
:1050B00006E061A000F016FD214660A0FEF7B0FA00
:1050C00000BF60E728736B697029000000000000D2
:1050D0005B434D445D20434D443D25732050313D9D
:1050E00025732050323D25732043533D25303258DF
:1050F0002F253032582025730D0A0000524C000035
:10510000504152414D0000005B434D445D20496ECB
:1051100076616C696420524C20706172616D3A2036
:105120006E6F74206E756D657269630D0A00000004
:10513000524C2C25640000004F4E00004F464600A4
:105140005B434D445D2052656C6179202D3E2025E6
:10515000730D0A005B434D445D20496E76616C69B6
:105160006420524C20706172616D3A2073746174D6
:10517000653D25640D0A0000444900003000000030
:1051800044492C2564256425642564005B434D4413
:105190005D20444920616C6C207374617465733ABE
:1051A000203078253032580D0A00000044492C2563
:1051B000642C2564000000005B434D445D2044499D
:1051C0002564203D2025640D0A0000005B434D440A
:1051D0005D20496E76616C69642044492063686192
:1051E0006E6E656C3A2025640D0A00005B434D44E9
:1051F0005D20496E76616C6964204449207061725B
:10520000616D3A206E6F74206E756D657269630D05
:105210000A0000004543484F000000005B434D4436
:105220005D204543484F20726573706F6E73652033
:1052300073656E740D0A0000434D44005B434D449A
:105240005D20556E6B6E6F776E20636F6D6D616E56
:10525000643A2025730D0A0010B500200649087035
:1052600081F84E0081F84F0081F852004D2102482C
:10527000401CFAF78FFF10BD3402002000200349C4
:10528000086003490860034908607047A0000020D7
:10529000A4000020A8000020014611B96FF0020010
:1052A00070470248006808800020F9E7A800002045
:1052B00030B503460C460BB104B112B96FF00200D1
:1052C00030BD1448006818B900201080401EF7E770
:1052D00000201080002115E00F48104D2D68405D22
:1052E00058540E480068401CC0F309000B4D28605C
:1052F00008480068401E074D28601088401C108038
:10530000481C81B2A14203DA024800680028E3D1B8
:105310000020D5E7A800002034120020A4000020BF
:1053200030B502460B4602B113B96FF0020030BD32
:1053300000211AE00F480068B0F5806F02D34FF0EB
:10534000FF30F4E7505C0C4C0C4D2D6860550B4859
:105350000068401CC0F30900084C20600548006844
:10536000401C044C2060481C81B29942E2DB0020C2
:10537000DDE70000A800002034120020A00000207B
:105380000748006850B106480068401E044908609C
:105390000846006810B901200249087070470000F3
:1053A000B0000020B400002010B502210D48FCF729
:1053B000B1FAA0B9FCF7BCFA044607E0FCF7B8FA6A
:1053C000001B642802D36FF0010010BD02210548C4
:1053D000FCF7A0FA0028F1D00220FCF7F7F8002033
:1053E000F3E70000000C01400548007810B94FF0C9
:1053F000FF30704700200249087000BFF9E7000045
:105400009C00002010B5FFF739FF10BD10B5044611
:105410002046FFF741FF10BD70B504460D46164605
:10542000324629462046FFF743FF70BD0848007802
:1054300010B14FF0FF307047002006490860064960
:105440000860064908600120014908700020F2E761
:105450009C000020A0000020A4000020A800002044
:1054600070B50546FFF7A0FF04460CB1204670BD9D
:1054700035B1012D0FD0022D18D0032D2CD120E0F5
:10548000002280211C48FCF74DFA002201211B4814
:10549000FCF748FA23E0012280211748FCF742FA82
:1054A000002201211548FCF73DFA18E00022802176
:1054B0001148FCF737FA012211461048FCF732FA7E
:1054C0000DE0012280210C48FCF72CFA0122114644
:1054D0000A48FCF727FA02E06FF00200C7E700BFB6
:1054E0000520FCF773F8FFF75FFF04460CB1204678
:1054F000BDE70020BBE7000000080140000C0140B0
:1055000008B5094800684068C0B2009001216846AB
:10551000FFF706FF0A2005490860012204490248F6
:10552000FDF76AF908BD00005C010020B000002012
:10553000AC00002070B504460D4604B115B96FF0FB
:10554000020070BD4FF6FF732A4621460448FDF75E
:10555000A9F9064616B16FF00100F2E70020F0E766
:105560005C01002070B505461348007810B14FF07B
:10557000FF3070BDFFF75AFF044614B14FF0FF3003
:10558000F7E735B90D480E490A68026009790171DB
:1055900004E00A482968016029790171074800F090
:1055A000F1F804461CB1FFF71FFF2046E1E7012098
:1055B000014908700020DCE78C0000208D000020ED
:1055C000B65D000870B5054615B94FF0FF3070BDE7
:1055D00028210F48FAF7DEFD00200D49087081F8F8
:1055E0002500084629680162297980F824102030B6
:1055F00000F0C8F804460CB12046E8E7002000F0AF
:10560000EDF804460CB12046E1E70020DFE700009A
:10561000C00000202DE9F04104460D4616461F4605
:1056200014B10DB106B11FB94FF0FF30BDE8F081E4
:105630000A2D02DA4FF0FF30F8E72078542802D123
:105640006078582802D04FF0FF30EFE73B463246F3
:1056500002A1E01CFAF7CEFD0020E7E725642E2525
:10566000642E000010B500F05DF804460CB1204631
:1056700010BD01200249087081F825000020F7E7DD
:10568000C000002010B594B0254890F8250008B956
:1056900014B010BD2248007820B1012806D002289D
:1056A00036D134E001201E49087035E00020039017
:1056B00003A904A800F02AFB40B300200290019047
:1056C000039881B201AB02AA04A8FFF7A3FF044626
:1056D000DCB913484068401C114948600298886151
:1056E000019848610846C0690199884202D20C4974
:1056F0000198C86100F074F9012000F03DF93220F2
:10570000FBF764FF002000F037F900BF04E003E07E
:1057100002200349087000BF00BF00BFB8E70000C7
:10572000C000002010B50C48007810B96FF00500DB
:1057300010BD0A48007810B16FF00100F8E7FFF7DC
:1057400061FE044614B14FF0FF30F1E70120034938
:1057500008700020ECE700008C0000209200002080
:1057600010B50446C0200649087008462168C0F8F4
:105770000110217941710621FFF7DCFE10BD000008
:10578000340E002070B5054615B96FF0030070BDEA
:10579000FFF70AFE044614B16FF00200F7E703209A
:1057A000FFF75EFE044614B16FF00200EFE72846F3
:1057B000FFF7D6FF6420FBF709FF0020FFF750FE3C
:1057C000044614B16FF00200E1E703482968016064
:1057D000297901710020DAE78D00002070B50446B8
:1057E0002046FFF73DFE054615B16FF0020070BD83
:1057F0000020FCE770B505460E4605B116B96FF0FE
:10580000030070BD0848007810B96FF00500F8E794
:1058100031462846FFF78EFE044614B16FF00200B1
:10582000EFE70020EDE700008C00002070B5054692
:1058300015B94FF0FF3070BD1C210E48FAF7AAFCD5
:1058400000200C490870487608462968416129798A
:1058500001761430FFF796FF04460CB12046EAE7C4
:105860000020FFF7BBFF04460CB12046E3E7002011
:10587000E1E70000E8000020024602B111B94FF054
:10588000FF307047064882600020054B586018467C
:10589000C160002018611870012058760020F0E7E0
:1058A000E800002070B588B03248407E08B908B0E2
:1058B00070BDFCF73DF804462E48007830B1012851
:1058C00008D0022842D003284CD14AE001202949BF
:1058D00008704BE02748406826498968884206D30B
:1058E000032024490870002000F0CCF93EE0214854
:1058F0000069201A1F49C968884226D31D4840689C
:10590000431C1C4820218268684600F063F9054664
:10591000002D16DD29466846FFF76CFF06467EB966
:1059200014484068401C134948600846046101203F
:1059300000F0A8F93220FBF749FE002000F0A2F9A0
:1059400000BF02200B49087000BF0FE00948006942
:10595000201A0849C968884202D301200549087005
:1059600004E003E003200349087000BF00BF00BF4C
:105970009DE70000E800002010B5044614B1FFF7D1
:105980004FF901E0FFF742F910BD002120F8801F18
:1059900041808180C1808038704710B50246012364
:1059A00072B6B2F88400802806DBB2F88600401C8C
:1059B000A2F88600002310E0B2F88000115432F8FB
:1059C000804F601CC41700EB5464E411A0EBC414B6
:1059D00014809088401C9080803A62B6184610BDB2
:1059E0000D48C069B8B10C48C0690B494968411AF3
:1059F0000948C160C06958B10748C068642148437C
:105A00000549C969B0FBF1F0C1B20348017402E075
:105A10000021014801747047C0000020F0B589B032
:105A200004460D46631C19A2202101A80095FEF72B
:105A300051FB0646701EC1B20DF10500FFF72DF8AF
:105A40000746C6F1200101AA90193B4614A2FEF7B1
:105A500041FB0DB114A000E015A00246611C15A089
:105A6000FDF7DEFD01A90020FDF76CFA01A916A0E3
:105A7000FDF7D6FD1A48006828B101AA294620463C
:105A8000174B1B68984709B0F0BD00002444495FDC
:105A90004556454E542C25642C25642A00000000F0
:105AA000253032580D0A00004849474800000000E0
:105AB0004C4F57005B494F5D2043482564202D3EE5
:105AC0002025730D0A0000005B494F5D20524634CB
:105AD00033332054583A20222573220D0A00000047
:105AE0005800002070B588B005462B4611A2202131
:105AF0006846FEF7EFFA0446601EC1B20DF10100E0
:105B0000FEF7BEFF0646C4F120010DEB040033464C
:105B10000BA2FEF7DFFA0C48006830B169460B486B
:105B20000078094A1268904702E06846FDF7F2FDE6
:105B300008B070BD244552522C25732A0000000085
:105B4000253032580D0A0000080000200C0000200B
:105B500070B590B005462B4611A240216846FEF76D
:105B6000B9FA0446601EC1B20DF10100FEF788FFCC
:105B70000646C4F140010DEB040033460AA2FEF7CD
:105B8000A9FA0B48006830B169460A480078084A0B
:105B90001268904702E06846FDF7BCFD10B070BD8A
:105BA000244F4B2C25732A00253032580D0A000053
:105BB000080000200C00002010B500F0CFF80448C9
:105BC000006820B102480068401E0149086010BD0D
:105BD000000000202DE9F84305460E46174698467A
:105BE0000DB1102E02DA0020BDE8F8833B4607A273
:105BF00031462846CDF80080FEF76CFA0446002CAA
:105C000001DDA0B2F0E70020EEE7000054582E2599
:105C100030336C752E2530336C752E00F8B5054683
:105C20006B206843164901EB800606F190040027BB
:105C300072B694F80601D0B9B4F80401002816DD54
:105C4000B4F80201205C009004F581742188481C9E
:105C5000C11700EB11610912A0EB012121806088BE
:105C6000401E608001202071A4F58174012762B676
:105C700027B1012269463068FCF76DFEF8BD0000CF
:105C80006C06002010B5044614B1FEF7DDFF01E0FC
:105C9000FEF7D0FF10BD002100F58070018041802B
:105CA000818081710181A0F58070704770B50346D5
:105CB0000C46002572B6002021E0B3F80411FF293C
:105CC00005DDB3F80811491CA3F8081119E0215C9F
:105CD000B3F800619955B3F80061711CCE1701EB60
:105CE00016663612A1EB0626A3F80061B3F804117C
:105CF000491CA3F80411691C8DB2411C88B2904262
:105D0000DBDB00BF62B6284670BD0000F8B5064672
:105D10000D4606B10DB90020F8BD0F48007808B94E
:105D20000020F9E76846FFF771FB04460CB100203C
:105D3000F2E7BDF8000008B90020EDE72A46FF2190
:105D40003046FFF769FB04460CB10020E4E7002071
:105D5000014908700120DFE7B400002000B5FFF71B
:105D60000FFB00BD6C5E0008645E00085C5E00080E
:105D7000745E00085C010020A4010020EC010020FA
:105D80007C5E0008845E00088C5E00080203040547
:105D9000060708090A0B0C0D0E0F10100102000077
:105DA00000000000000001020304060708090000CB
:105DB00000000102030400001A1704C1C1C14154CC
:105DC0002B444556545950453D3F0041542B4657AE
:105DD000434F44453D3F000040404040404040402C
:105DE00040414141414140404040404040404040AE
:105DF0004040404040404040050202020202020290
:105E00000202020202020202202020202020202082
:105E100020200202020202020290909090909010C4
:105E20001010101010101010101010101010101072
:105E300010101002020202020288888888888808EE
:105E400008080808080808080808080808080808D2
:105E50000808080202020240D85D00085741524E6D
:105E600020000000494E464F2000000044454255A6
:105E7000470000004552524F520000005541525415
:105E80003100000055415254320000005541525437
:105E900033000000B45E000800000020C0000000D5
:105EA0007C410008745F0008C000002078190000E1
:105EB0008C4100080000000000000000000000000D
:105EC00000000000000C0140100000000000000075
:105ED00000000000000C0140200000000000000055
:105EE00000000000000C0140400000000000000025
:105EF00000000000000C01408000000000000000D5
:105F00000000000000000000010000000000000090
:105F10000000000000000000000000000000000081
:105F20000000000001000000000000000000000070
:105F30000000000010000000010000000024F40038
:105F40000000000000000000000000000000000051
:105F50000000000000000000000000000000000041
:105F60000000000000000000000000000000000031
:045F7000000000002D
:04000005080000ED02
:00000001FF
